:030000000219FDE5
:03000B000200AA46
:03002B0002015C73
:03005B000202EEB0
:030073000202DBAB
:1000800002030406080C10182030406080040608A3
:100090000C10182030406080A0C00003070F1F0D17
:1000A0000D0403060D0503030202C2AFC0D0C0E079
:1000B000206214E5256009E473E525F4F58AD2622F
:1000C000D0E0D0D0D2AF3285268AC262E526F46075
:1000D0002F30682520720DD0E0D0D0C295C293C2D7
:1000E00097D2AF32C295C293C297206F0C20650998
:1000F0007409D5E0FDE57B4290D0E0D0D0D2AF329C
:10010000758A00C28DD26201F901B9306805206597
:1001100002D29501B9306805206502D29701B93045
:100120006805206502D29301B9C29430680A20653F
:10013000077409D5E0FDD29501B9C29630680A204E
:1001400065077409D5E0FDD29701B9C29230680AFB
:100150002065077409D5E0FDD29301B9C2AFC2ADE5
:1001600053E6EFC0D0C0E0D2D3D2AFC2CEE52A6012
:100170000720744F152A21C37800790020742EE5DA
:1001800080307E01F430E50278FF53DACF207E0321
:1001900043DA20307E0343DA10C2D8C271E58030E2
:1001A0007E01F430E50279FFC3E89970CB3061033A
:1001B000752A40207403752A40885CD270E8600379
:1001C000755F0020740DE52B6004152B21D343DAF5
:1001D00001C2D820700221E6A85C206102C2702012
:1001E000740221E488227882B6040385222420CF79
:1001F0000AD0E0D0D043E610D2AD32C2CF053A7873
:1002000002E52A6005307402152AC3E55C940140BA
:1002100005755F004127756000756900E55F240181
:10022000F55F5003755FFF7982B7020D306E1DC315
:10023000E52294324016854C227982B7030E306E47
:100240000BC3E52294324004798E8722C3E52395BF
:1002500022600840041523415B0523D8CA0569E5DF
:100260006970021569D56A69756A017808E56B607D
:10027000497805C3E569956B4057C3E569956C50AE
:10028000087801756A03020295C3E569956D50050A
:100290007801756A01C3E5629524401E7982B7042E
:1002A0000241C6206E14852462E569046003856BF3
:1002B00069756A0175233C0202D1E5622850057513
:1002C00062FF41C6F562E5620470067560FF7569FC
:1002D000FFD0E0D0D043E610D2AD32C2AF53E67FBC
:1002E0007592FA7593FFC260759104D2AF32C2AFB6
:1002F00053E6EFC2ADC0D0C0E0C0F0D2D3D2AFA8B9
:10030000FBA9FCC2D8307102615553DACF207E03BD
:1003100043DA10307E0343DA20D271E580307E016B
:10032000F420E502612C88278928A13A53DACF20EE
:100330007E0343DA20307E0343DA10C2D8C2713024
:100340007402A1267800E580307E01F430E502A138
:1003500026885CA10E53DACF207E0343DA20307E5C
:100360000343DA10C271206102812E53DACF207E5E
:100370000343DA10307E0343DA20C2D8D2718857A3
:100380008958C3E89555F8E99556F97B007E087AB7
:1003900000C3E8948CE994005005755B00812088C7
:1003A0002178A2E6A8216055C3E894C8E9940050DA
:1003B00008E4D2E4FB7A0A61FBC3E89468E994019B
:1003C0005008E4D2E3FB7A0F61FBC3E894D0E994D0
:1003D000025008E4D2E2FB7A1E61FBC3E894A0E974
:1003E00094055008E4D2E1FB7A3C61FBC3E89498A1
:1003F000E994085008E4D2E0FB7A787E00C3E895DF
:1004000059FCE9955AFD30E70AECF42401FCEDF4BF
:100410003400FD755B00C3EC9AED9E5003755B01E3
:100420008859895A8557558558567802A10EC3E8D0
:100430009527F8E99528F9307C0281F2307B02811A
:10044000F2307A0281EB2075028151E9FDE8FC81EE
:1004500070E9C313F9E813F830790281EBE9C313AB
:10046000F9E813F830780281EBE9C313FDE813FCD7
:0F04700020612CC3EC941CED940240028187EDB7
:10047F00701EC3EC94C850180529E5297002152980
:10048F00C3E529940A5002A126755C00D270A126FB
:10049F00E529600215297400207F037896E624FA77
:1004AF00FEE43400FFC3EC9EFCED9FFD5006780088
:1004BF00790081F2C3EC94FFED9400400678FF7948
:1004CF000081F2EC8572F0A4C5F0A2F733F8790041
:1004DF00400302050E78FF790002050EE9C313F9F8
:1004EF00E813F8307C0EE9600278FFC3E81338F8A0
:1004FF00E43400F9C3E894FFE99400400278FF88E0
:10050F005CD270206102A126741FF4552F4BF52F7A
:10051F00C274EB7002D274752A40307403752A0AC4
:10052F00306102A13A20740353DAFE207403752B55
:10053F0020D0F0D0E0D0D0D2AD43E6103279010216
:10054F00056A790302056A790A02056A791E0205AE
:10055F006A796402056A79C802056A7817E4D5E0FA
:10056F00FDD8FAD9F6227A147B780205917A107B9E
:10057F008C0205917A0D7BB40205917A0B7BC80230
:10058F000591E573D5E001227902E4C296D5E0FD2D
:10059F00D297D5E0FDC297D5E0FDD296D5E0FDE923
:1005AF0020E002D29530E002D293E573D5E0FDE969
:1005BF0020E002C29530E002C2937496D5E0FDD9D7
:1005CF00C9EAF8D5E0FDD8FBDBB8C29622C37C00A0
:1005DF007D0075F00005F0EA33FAEB33FB50F6EBD4
:1005EF0013FBEA13FAC3E9FFE8FEE89AF8E99BF96F
:1005FF005004EFF9EEF8B3EC33FCED33FDD5F0DF3B
:10060F00EDF9ECF822E889F08A20D2D4F8A9F07B32
:10061F000030F70B7BFFF42401F8E9F43400F9E81C
:10062F008520F0A4ADF0F8E98520F0A4AFF0FEED41
:10063F002EF974003FFA7C04C3EA13FAE913F9E8C0
:10064F0013F8DCF48BF030F70AE8F42401F8E9F43E
:10065F003400F9E889F0C2D4F8A9F0227882B60400
:10066F000302070AC3E55C9419401EE52D5406707A
:10067F0018206E3678057994E7146007780A1460AD
:10068F00027812C3E54198401F306E098564627588
:10069F0069FF756A01852224E4F544F545F546F5B1
:1006AF0047F548C26E02070AD26E7994E7147013A9
:1006BF00E523F43333F913F8E9540104F9E854FE50
:1006CF000206FEE714147014E523F4333333F913E1
:1006DF00F8E9540304F9E854FC020706E523F43360
:1006EF00333333F913F8E954070404F9E854F8C322
:1006FF009440F8E99400F98844894522C3E54113F1
:10070F00F9E54013F8C3E54498F8E54599F9500C1D
:10071F00C3E89480E994FF4016020742C3E8947F30
:10072F00E994005003020742787F7900020742786C
:10073F008079FF8849894A22E5492546F8E54A35F7
:10074F0047F9854A20E4300701F43548FA30E709C4
:10075F00C3EA94F04015020780C3EA940F500302D6
:10076F00078078FF79FF7A0F020780780079007A87
:10077F00F0C3E5249561500AC374019524500B0210
:10078F00079EE54A20E70E02079EE54A30E70688F6
:10079F004689478A482278A5E6FAC3E54933F8E542
:1007AF004A33F9D114E930E70BC3E89480E994FF99
:1007BF004013E1D8C3E8947FE994005002E1D87860
:1007CF007F7900E1D8788079FFE820E715C3E5232A
:1007DF0098F84009C3E8940140030207FF7801022B
:1007EF0007FFE8F424012523F840030207FF78FFF1
:1007FF00884B2278A6E6FAA847A948120614E930D2
:10080F00E70CC3E89401E994FF4016020834C3E8EB
:10081F0094FFE99400500302083478FF790002082E
:10082F0034780179FFE920E715C3E54B98F84009C3
:10083F00C3E89401400302085B780102085BE8F407
:10084F002401254BF8400302085B78FF88242278A7
:10085F00FF20692879A1E76023E541601F74FF85B8
:0E086F0041F0848539F0306A0375F005A4F875
:10087D00C5F0600278FFC3E895645002A8648863F0
:10088D0022C3E5409440E5419401E5635003140112
:10089D009F046002F563227883E6F520120F297517
:1008AD00E89012054C75E89030EDFDA8BDA9BE127B
:1008BD000FD4756E2B756F00C3740013FD742B6010
:1008CD006613FC742B2CFC74003DFDECFAEDFBC3A0
:1008DD00E89AE99B4014E56E242BF56EE56F340024
:1008ED00F56FEA2CFAEB3DFB80E5AE6EAF6FC3E51D
:1008FD006F13F9E56E13F8C3E913F9E813F87A03EA
:10090D00C3E913F9E813F8DAF7AA201A7009756E1E
:10091D0000756F000209341AEA6008EE28FEEF39FF
:10092D00FFDAF88E6E8F6F2275E890227883E6FFDE
:10093D0030EDF9A8BDA9BE0570C3E570940840520D
:10094D00757000E9FA79A0E76044EA7007E5716017
:10095D001B02096DC3E895716010E5715006600CBE
:10096D00140209790460F9020979E571F571C394EE
:10097D006D401B7561C0C394044013756180C394B1
:10098D0004400B756140C39404400375610075BB51
:10099D000822EFC39401601F742B601BC3E894FF02
:1009AD00E994035012C3E8956EE9956F5009E5611E
:1009BD00600C15610209CBE561F460020561A86167
:1009CD00C3E524985002A824C3E89562400AA862A2
:1009DD00E562F4600385626188258826E570B407B9
:1009ED000375BB1022743279A787F0A4C5F0A2F766
:1009FD0033F8C3E895614002A861882288248825D0
:100A0D0088268864227540007541F022C2AF75C8F2
:100A1D0020A8CCA9CDAA3A30CF010A75C824D2AFEF
:100A2D00AB3BAC3C883B893CC3E89BF8E99C206917
:100A3D0008F9306602612A4184AD3D8A3DF9EA9D8F
:100A4D00FA600678FF79FF4169AE3EAF3F8B3E8C71
:100A5D003FA83BA93CC3E89EF8E99FF9C3E54113C4
:100A6D00FBE54013FAE82AF540E93BF541500675E0
:100A7D0040FF7541FF41D1AA40AB41AC40AD417E35
:100A8D00047F02C3EB9404400D1E1FC3EB9408407A
:100A9D0005206A021E1FC3ED13FDEC13FCDEF7C328
:100AAD00EA9CFAEB9DFBEF6009C3E913F9E813F833
:100ABD00DFF7EA28FAEB39FB8A408B4150067BFFC2
:100ACD008B408B41C3EB94025002D2663069047F98
:100ADD000341FC7892E6FFC3E537948240110FC3C2
:100AED00E53794A040010FC3EF940640027F057EC9
:100AFD0002E541C4540FF9E541C454F0F8E540C492
:100B0D00540F28F8C3E89EFAE99400FB4009C3EAA4
:100B1D009402EB940050047A02E4FB6176AA40AB98
:100B2D0041EBC4FEEAC4540F4EFCC3EA9CFAEB94AD
:100B3D0000FBC3E813C313F8EA28FAEB3400FB8A71
:100B4D00408B41C3EB94024002C2667802EBC4FEB7
:100B5D007B00EAC4540F4EFAC3EA98FA4005C394D9
:100B6D000250027A027892E6FF306002617685517A
:100B7D0092855293D26043E680C3E49AF8E49BF9E0
:100B8D003066028102E8FAE9FBD3E913FDE813FCB4
:100B9D0088518952C3EF94036038EF20E00DE82CA3
:100BAD00F8E93DF9ECFAEDFB020BCBE828F8E93951
:100BBD00F9C3E82402F8E93400F97AFE7BFFC3EFAC
:100BCD009403400E8A538B54884D894E8C4F8D5013
:100BDD008136885389548A4D8B4E8C4F8D50306998
:100BED00127553F07554FF754FF07550FF7551F038
:100BFD007552FF8136E8FAD3E813FC8851C3EF94A0
:100C0D00036020EF20E007E82CF8ECFA8122E828B9
:100C1D002402F87AFEC3EF940340088A53884D8C62
:100C2D004F813688538A4D8C4FE568C3335002642B
:100C3D006BF5683060028140753402D26043E68006
:100C4D00E52D54066034A840A941C3E913F9E81312
:100C5D00F8C3E913F9E813F8306904E92440F9C23F
:0E0C6D00AF53E67F759100C3E498F594E499C7
:100C7B00F595759104D26043E680D2AF22D26475AC
:100C8B004300752000306C03752040020CA7D26422
:100C9B00754300752040306C037520007801790195
:100CAB00206620E52D54066002C2647914E541C329
:100CBB0013700104F8C3941440027814306904785B
:100CCB001B791B206010E543600C306903D534049D
:100CDB00D26DA15191480543E59B5440B52002A12B
:100CEB003B30690908C3E89940011881CE20640A9A
:100CFB0008C3E899400281A781CEC264C2AF53E614
:100D0B007F7591003066127594007595F875910496
:100D1B00D26043E680D2AF81A7E5417EFFC333406B
:100D2B0005C3334001FEC3E49E759400F595A118ED
:100D3B00C3E5339401500281A730640281A7D80226
:100D4B00A14F81CEC26DC2AF53E67F759100855323
:100D5B0094855495759104854D92854E93D260433D
:100D6B00E680D2AFE52D54066008206A02053302F7
:100D7B000D8D306D0D206C0A2064071581158102D5
:100D8B0016422278003064027801E53775F007A42B
:100D9B00F9E5F028F5F0E9A2F013A2F113A2F21392
:100DAB00F537C394785003753778C3E537953840DA
:100DBB0008D265C295C293C297306002A1C4854F19
:100DCB0092855093D26043E68022D281207D16C259
:100DDB00AF754202C296D294306202D293D2AF75F3
:100DEB009F11020FD1C2AF754202C296D2923062EE
:100DFB0002D295D2AF759F11020FD1C281307243CF
:100E0B00207D20C2AF75420390013A757B40C2939F
:100E1B00C292306204D297C126D296D2AF759F137D
:100E2B00020FD1C2AF75420390013A757B40C29558
:100E3B00C294306204D297C146D296D2AF759F103E
:100E4B00020FD1207D17C2AF754203900115C293DB
:100E5B00306202D297D2AF759F13020FD1C2AF751A
:100E6B004203900115C295306202D297D2AF759FA3
:100E7B0010020FD1D281207D16C2AF754204C294ED
:100E8B00D292306202D297D2AF759F10020FD1C2AD
:100E9B00AF754204C292D294306202D297D2AF7530
:100EAB009F13020FD1C281307243207D20C2AF75D8
:100EBB004205900129757B10C297C296306204D20D
:100ECB0095C1D0D294D2AF759F11020FD1C2AF751D
:100EDB00420590014B757B04C297C296306204D2D7
:100EEB0093C1F0D292D2AF759F11020FD1207D1713
:100EFB00C2AF75420590010BC297306202D295D2F8
:100F0B00AF759F11020FD1C2AF75420590011FC281
:100F1B00973062EBD293D2AF759F11020FD1D28172
:100F2B00207D16C2AF754206C292D296306202D2B3
:100F3B0095D2AF759F13020FD1C2AF754206C29403
:100F4B00D296306202D293D2AF759F10020FD1C2EC
:100F5B0081307244207D20C2AF75420190014B75E8
:100F6B007B04C295C294306204D293E17AD292D2BE
:100F7B00AF759F10020FD1C2AF7542019001297559
:100F8B007B10C293C292306205D295020F9BD29412
:100F9B00D2AF759F13020FD1207D17C2AF754201DF
:100FAB0090011FC295306202D293D2AF759F10028F
:100FBB000FD1C2AF75420190010BC293306202D2C6
:100FCB0095D2AF759F13C26522900109757B00C244
:100FDB0095C293C297C294C292C296C26222788083
:100FEB0076070876070876010876040876FF0876F8
:100FFB00FF087608087602087601087601788C7669
:10100B00010876000876B40876FF0876FF0876FFAD
:10101B000876030876FF0876010876FF0876250820
:10102B0076D00876780876C80876040876FF0876B6
:10103B000108760008767A087610087601087601A2
:10104B000876000876FF087600227887E6FFC272E2
:10105B00BF0302D2727888C27DE630E102D27DC234
:0F106B007E7889E630E102D27EC3EF94026008FE
:10107A00758E01D273021087758E00C27322788032
:10108A00E6149000809378A5F67881E614900080A3
:10109A009378A6F67886E61490008D9378A7F6786A
:1010AA009FE6F87005756B0001CEC3E89411400203
:1010BA007811E82828F56B256B256B28F56C256BCC
:1010CA002828F56D7886E6F539C3940250037539F8
:1010DA0002789CE67538FFB402037538A0B403039E
:1010EA0075388278A3E61490009A93F566120FD4A5
:1010FA0022227896E6FA7897E6FB7888E6B4030522
:10110A00C3EB940EFB307F047A007BFFC3EB9AFC9F
:10111A00C3948250027C827572000572EC8572F06B
:10112A00A4C3E5F0947D40F222D27F11FC12055B44
:10113A0012055B7A007B007C10120551E55C2AFAE5
:10114A0074003BFBDCF37C04C3EB13FBEA13FADC0D
:10115A00F7FEC27F11FC22757C00757D00E5EF2049
:10116A00E6037520000520903FFFE52014600690F5
:10117A001DFF1460009304600375EF1653D9BF7501
:10118A0081C043FF8012054C75EF0643B203E5B3F5
:10119A00240220E70DF521E5E320E0068521B3438B
:1011AA00E301120FD47580FF75A40275F1B275D4EC
:1011BA00DF75900175A5FC75F2FE75D50175A6015E
:1011CA0075E241120FD4E4F8F6D8FD756801120FE2
:1011DA00E912169978988673753001C2AF120565BF
:1011EA0012057512055B12057C12055B1205831246
:1011FA00055B1217CC120565120565120560C2AFB0
:10120A00757C00757D0078FA79FA308507D9FBD8A4
:10121A00F7021C001155118811FB11FC789886738E
:10122A00120FD475881075890275C82475910475D2
:10123A00D84075A82275B80275E690759B80759D91
:10124A000075D10E75BC5875BB0875BA1175E88062
:10125A0012054CD2AF1208A475360053DACF207E9D
:10126A000343DA20307E0343DA1043DA01C2D8C2DC
:10127A0071120565D2617B037A0CE55B70077A0C03
:10128A00DB0302120812055B207003021208C27007
:10129A00E55CC3940240E1E52F541F855E5DF55E6F
:1012AA00B55DD5DAD5C26153DACF207E0343DA20A1
:1012BA00307E0343DA10C2D8C27178A2E67008D22F
:1012CA0074E52F54E0F52FC27575290012056030B8
:1012DA007409C3E529940A4002D2751205517802AD
:1012EA003074027800C3E55C9840F0C2AF1205750D
:1012FA00120575120575D2AF120565754C001205F7
:10130A0051788CE6C3940150030213F5E530C39477
:10131A000150030213F5757CA5757DF1207435C360
:10132A00E55C94FF50030213F5C2AF12058AD2AFEF
:10133A00120560C3E55C940150EFC2AF1205751245
:10134A000556120575D2AF120560C3E55C94FF40DD
:10135A00E90218517F05D27F11FC120560C2AFC2A3
:10136A007F11FCAE5CC3E55C947FD2AF500281056D
:10137A0012054CC2AF12058AD2AFDFDA3133C3EE9F
:10138A0094057897F61205651217D47F0AD27F1151
:10139A00FC120560C2AFC27F11FCAE5CC3E55C946F
:1013AA007FD2AF50E612054CC2AF12057512055630
:1013BA00120575D2AFDFD63133EE24037896F6F8EC
:1013CA007997E7C394824003985006E82482789775
:1013DA00F61205651216E712180312056011FCC30E
:1013EA00E55C94FF50026120021851757C00757DFE
:1013FA0000C3E55C954C4003855C4C12056078019E
:10140A007988E7B403027805C3E55C98400261086D
:10141A00C2AF12058A12058A12058AD2AF12056571
:10142A00753000E4F531F5320531E531F4703F05E8
:10143A0032789AE67819146012783214600D787D41
:10144A0014600878FA146003753200C3E5329840D4
:10145A001D120FD412054C15327531007899867316
:0E146A00C2AF12058AD2AF7898867312056061
:10147800120556E52A700530740241087801207477
:10148800027806C3E55C9840A1120560E52A70035E
:10149800021208C2AF120FD4E4F522F523F524F5A1
:1014A80025F526F567D2AF7885E6C333F565E4F50B
:1014B80044F545F546F547F548F570F52CF52DF555
:1014C8003775700875BB1012054C12093530EDFDE3
:1014D800A8BDA9BEE97001F88871120939757008AC
:1014E80075BB101155C2AF7561FF1209F2852261F3
:1014F800852262852263D2AF752201752401752584
:1015080001752601856069756A017888E6B4030764
:10151800C27D307602D27DD268D269753300120F4F
:1015280029120F5A120A12120A19120A12120A1949
:10153800120A12120C9912066B120D8E120DD51288
:101548000A19120C88306E0312070B206603120862
:101558005E30660312088E120D8E120E06120A19DC
:10156800120C99306E03120747120D8E120E7F125D
:101578000A19120C88306E031207A5120D8E120E6E
:10158800B0120A19120C99306E03120802120D8E4D
:10159800120F29120A19120935120C88120D8E120F
:1015A8000F5A120939120A1930692C856461856449
:1015B80062856069756A0179187A0CC3E5339940C8
:1015C80009C269D26A8A350215DFC3E55C94014015
:1015D8000302153B02164A306A25206C22E53514B1
:1015E8007006C26AD26BA13BF535C3E55C94014035
:1015F8000302153B7888E6C39403600302164A7514
:101608003600C3E55F9401400985646285606975A9
:101618006A0178FA79A4E760027803C3E55F985015
:1016280021307404E52A601A78F0306C058564610D
:101638007820C3E541985002A13B0536E55C60027D
:10164800C14D753600C2AF120FD47887E6FE760218
:1016580011557887EEF6E4F522F523F524F525F5FE
:1016680026F565752C00752D00D2AF120560120F96
:10167800D478A4E66006D295D297D293307406E562
:101688002A70024108788DE6C39401400241E58141
:101698002D901A0D7820121729E520B4A50CA31255
:1016A8001729E520B45A030216C7757CA5757DF184
:1016B800120FE91216E7757C00757D000216E69098
:1016C8001A0378807B0A121729A308DBF9901A0FEE
:1016D800788C7B19121729A308DBF9901A2822C2E3
:1016E800AF12176C121749901A00740E12172EA316
:1016F800740912172EA3741512172E901A037880E6
:101708007B0A12172DA308DBF9901A0F788C7B1926
:1017180012172DA308DBF912177F12175D901A28EC
:1017280022E493F622E6438F01538FFDFFC3E5833E
:10173800941C400122EF857CB7857DB7F0538FFE5E
:1017480022438F02438F01857CB7857DB7901A0DA0
:10175800F0538FFC22901A0D74A5F12E901A0E7476
:101768005AF12E227A3079D07820901A40F129E562
:1017780020F709A3DAF7227A3079D0901A40E7F1F6
:101788002E09A3DAF922AB74A875BB01027980BBD4
:1017980002027981BB03027982BB04027994BB05FA
:1017A800027983BB06027986BB07027992BB0802DD
:1017B8007987BB0902799CBB0A027988BB0B02793D
:1017C80089E8F7227C05120565DCFB22C2AF120509
:1017D8007512057C12058312058A120556120575C5
:1017E80012057C12058312058A1205561205751218
:1017F800057C12058312058AD2AF22C2AF12058A70
:1018080012058312057C12057512055612058A12F7
:10181800058312057C12057512055612058A1205F4
:101828008312057C120575D2AF22AE74AF75C2AFB4
:10183800120575120575120575120556DEF21205A8
:101848008A120556DFF8D2AF221217D41217CC121B
:1018580017CC75740175750175760011327C05AD6C
:0F1868005C120565C3ED955C70F5C3E55C9401FA
:10187700400AC3E55C94FF403702189412178E1292
:1018870016E71217D4C2AF75EF161217CCDCD105C5
:1018970076C3E5769403500280C21217CC0575E52E
:1018A700741490009F93F808C3E57598500280A9B7
:1018B7001217CC1217CC0574C3E574940C50028030
:0F18C70095120FE91216E7C2AF75EF161217CC84
:0319FD0002116173
:101A00000E091507070104FFFF08020101A55A018D
:101A100000B4FFFFFF03FF01FF25D078C804FF01DA
:091A200000FF10010100FF00FFAE
:101A400023534B4D6F6E73746572383041232020E1
:101A500023424C48454C4923463333302320202031
:101A60002020202020202020202020202020202076
:101C0000C2AFC2D353D9BF7581C043B20343FF8073
:101C1000752438752503B1DC7529A5752AF175E29F
:101C20004043F12053A4DF75D4FFD2857DFA7803B9
:101C300079E67C10752200752300901DE97B0675FE
:101C400024987525013085028145208508D8FBD967
:101C5000F9DCF781B7308508D8FBD9F9DCF781B713
:101C6000B19CE493A3C39A6004DDC381B7DBDBB10D
:101C70008E6002812E7B08E493FAA3B16FDBF87AC1
:101C800030B16F752200752300B18EEAFCEBFDC305
:101C9000ED94FE400EB18E8A278B28ED30E0048A49
:101CA000828B83B18E7AC270D8C3ED94FE601950D6
:101CB000CEBD002BEC600F7520007521FF7529004B
:101CC000752A000200008100A827A9280809D80465
:101CD000D90281DCB192EA89AAF281CE0D81A3C337
:101CE000ED94035053EDA2E092007AC5C3E58294CF
:101CF00000E583941C508A200010438F02438F011B
:101D00008529B7852AB7F0300029A827A92808090E
:101D1000438F01538FFDD804D902A133C3E58394C7
:101D20001C4003A3A11689AAE28529B7852AB7F02A
:101D3000A3A116538FFC817F7AC1BD030CE493A34A
:101D4000FAB153DCF8B14B817F8181AA22AB23B178
:101D50006FEBFAEA6222752608C3E52313F523E543
:101D60002213F52250066323A0632201D526EAB18F
:101D7000DCB1DC75260AEAF4200102D285300102CA
:101D8000C285B1DCC3134002C201D526EB22B19259
:101D9000EAFB208502A192308502A197752608AE44
:101DA00024AF25C3EF13FFEE13FEB1E0B1DCC3EAAD
:101DB000133085024480FA30E703632201C3E52330
:101DC00013F523E52213F52250066323A0632201B5
:101DD000D526D9E52265236523F52222AE24AF2539
:101DE0000E0FDEFEDFFCD20122424C48656C6934E6
:071DF000373164F3300601F6
:00000001FF
